:100000000C945B000C94E8000C9415010C94830094
:100010000C9483000C9483000C9483000C94830054
:100020000C9483000C9483000C9483000C94830044
:100030000C9483000C9483000C9483000C94830034
:100040000C9442010C9483000C9487020C9483005E
:100050000C9483000C9483000C9483000C94830014
:100060000C9483000C948300000024272A000025B0
:10007000282B000023262904040404040404040299
:100080000202020202030303030303010204081035
:100090002040800102040810200102040810200002
:1000A0000000070002010000030406000000000039
:1000B00000000000DD0011241FBECFEFD8E0DEBF3E
:1000C000CDBF11E0A0E0B1E0E6EEF5E002C00590A2
:1000D0000D92AC30B107D9F711E0ACE0B1E001C04E
:1000E0001D92A23AB107E1F710E0C6EBD0E004C0E0
:1000F0002297FE010E94ED02C43BD107C9F70E947E
:10010000D6000C94F1020C94000061E08091000193
:100110000E94340260E47CE980E090E00E94B20139
:1001200061E0809102010E94340268E97AE380E094
:1001300090E00E94B20160E0809100010E943402D0
:1001400060E375E780E090E00E94B20161E0809199
:1001500000010E94340261E0809104010E94340297
:1001600068E97AE380E090E00E94B20160E080916B
:1001700000010E94340260E0809102010E9434027A
:1001800060E0809104010E943402089561E0809152
:1001900000010E94160261E0809102010E94160295
:1001A00061E0809104010E94160208950E94DC0122
:1001B0000E94C6000E948500FDCF8AE091E09093E6
:1001C0000D0180930C010895862F0E947F020895EF
:1001D0001F920F920FB60F9211242F933F934F93BC
:1001E0005F936F937F938F939F93AF93BF93EF939F
:1001F000FF9380910E0190910F01892B29F0E091DE
:100200000E01F0910F010995FF91EF91BF91AF9110
:100210009F918F917F916F915F914F913F912F911E
:100220000F900FBE0F901F9018951F920F920FB650
:100230000F9211242F933F934F935F936F937F936C
:100240008F939F93AF93BF93EF93FF938091100190
:1002500090911101892B29F0E0911001F091110189
:100260000995FF91EF91BF91AF919F918F917F91F0
:100270006F915F914F913F912F910F900FBE0F9013
:100280001F9018951F920F920FB60F9211242F9363
:100290008F939F93AF93BF9380911201909113011D
:1002A000A0911401B09115010196A11DB11D80937B
:1002B000120190931301A0931401B0931501809142
:1002C000160190911701A0911801B0911901805069
:1002D000904CAF4FBF4F8093160190931701A0939E
:1002E0001801B093190127C0809116019091170150
:1002F000A0911801B091190180589E43A040B040D0
:100300008093160190931701A0931801B0931901DF
:1003100080911A0190911B01A0911C01B0911D01C7
:100320000196A11DB11D80931A0190931B01A0930A
:100330001C01B0931D018091160190911701A091AD
:100340001801B091190181589E43A040B04060F659
:10035000BF91AF919F918F912F910F900FBE0F90F2
:100360001F901895EF92FF920F931F937B018C01C2
:100370008FB7F89440911A0150911B0160911C01B4
:1003800070911D018FBF2FB7F89480911A01909141
:100390001B01A0911C01B0911D012FBF841B950B67
:1003A000A60BB70BE816F9060A071B0760F71F91A3
:1003B0000F91FF90EF900895789484B5826084BD8A
:1003C00084B5816084BD85B5826085BD85B5816059
:1003D00085BDEEE6F0E0808181608083E1E8F0E0B9
:1003E000808182608083808181608083E0E8F0E0AA
:1003F000808181608083E1EBF0E080818460808394
:10040000E0EBF0E0808181608083EAE7F0E08081CA
:10041000846080838081826080838081816080832A
:100420008081806880831092C1000895282F30E079
:10043000C90185579F4FFC01949129583F4FF901FD
:100440008491882381F0E82FF0E0E859FF4FE49190
:10045000F0E0662329F480819095892380830895B4
:100460008081892B80830895482F50E0CA018156EE
:100470009F4FFC012491CA0185579F4FFC01949125
:1004800049585F4FFA0134913323C1F1222331F1EE
:10049000233021F4809180008F7705C0243031F41F
:1004A000809180008F7D8093800018C0213019F4E6
:1004B00084B58F7704C0223021F484B58F7D84BD4C
:1004C0000DC0263021F48091B0008F7705C0273011
:1004D00029F48091B0008F7D8093B000E32FF0E08D
:1004E000E359FF4FE491F0E0662329F48081909571
:1004F0008923808308958081892B80830895982F94
:100500008091C00085FFFCCF9093C60008951F9294
:100510000F920FB60F9211242F933F934F935F9337
:100520006F937F938F939F93AF93BF93EF93FF93BB
:100530004091C600E0911E01F0911F01CF0101968C
:1005400060E870E00E94C4029C01809120019091BB
:1005500021012817390739F0EE5DFE4F40833093B3
:100560001F0120931E01FF91EF91BF91AF919F91C9
:100570008F917F916F915F914F913F912F910F904C
:100580000FBE0F901F90189597FB092E07260AD0D3
:1005900077FD04D00CD006D000201AF47095619538
:1005A0007F4F0895F6F7909581959F4F0895AA1B68
:1005B000BB1B51E107C0AA1FBB1FA617B70710F04E
:1005C000A61BB70B881F991F5A95A9F78095909580
:1005D000BC01CD010895EE0FFF1F0590F491E02DB1
:0605E0000994F894FFCF1E
:0C05E600080009000A0000000000E4000A
:00000001FF
